:100000000C947D030C94A5030C94A5030C94A503F8
:100010000C94A5030C94A5030C94A5030C94A503C0
:100020000C94A5030C94A5030C94BF080C942E0902
:100030000C94A5030C94A5030C94A5030C94A503A0
:100040000C94A5030C94A5030C94A5030C94A50390
:100050000C94A5030C94A5030C94A5030C94600BBD
:100060000C94A5030C94A5030C94A5030C94A50370
:100070000C94A5030C94A5030C94A5030C94A50360
:100080000C94AA0B0C94A5030C94A5030C94A50343
:100090000C94A5030C94A5030C94A5030C94A50340
:1000A0000C94A5030C94A5030C94A5030000000078
:1000B000003E5B4F5B3E3E6B4F6B3E1C3E7C3E1CEE
:1000C000183C7E3C181C577D571C1C5E7F5E1C0034
:1000D000183C1800FFE7C3E7FF0018241800FFE7EB
:1000E000DBE7FF30483A060E2629792926407F05AE
:1000F0000507407F05253F5A3CE73C5A7F3E1C1CC4
:1001000008081C1C3E7F14227F22145F5F005F5F83
:1001100006097F017F006689956A6060606060946F
:10012000A2FFA29408047E040810207E2010080874
:100130002A1C08081C2A08081E101010100C1E0C7F
:100140001E0C30383E3830060E3E0E060000000011
:100150000000005F00000007000700147F147F14F8
:10016000242A7F2A1223130864623649562050003D
:1001700008070300001C2241000041221C002A1C29
:100180007F1C2A08083E0808008070300008080814
:100190000808000060600020100804023E51494534
:1001A0003E00427F400072494949462141494D3352
:1001B0001814127F1027454545393C4A49493141B9
:1001C000211109073649494936464949291E000087
:1001D00014000000403400000008142241141414DC
:1001E0001414004122140802015909063E415D59C8
:1001F0004E7C1211127C7F494949363E41414122D1
:100200007F4141413E7F494949417F090909013EFA
:10021000414151737F0808087F00417F4100204021
:10022000413F017F081422417F404040407F021C33
:10023000027F7F0408107F3E4141413E7F0909094A
:10024000063E4151215E7F09192946264949493216
:1002500003017F01033F4040403F1F2040201F3FDC
:100260004038403F63140814630304780403615961
:10027000494D43007F4141410204081020004141A3
:10028000417F04020102044040404040000307084F
:100290000020545478407F2844443838444444284B
:1002A000384444287F385454541800087E090218F2
:1002B000A4A49C787F0804047800447D400020407A
:1002C000403D007F1028440000417F40007C0478BE
:1002D00004787C080404783844444438FC18242406
:1002E0001818242418FC7C08040408485454542486
:1002F00004043F44243C4040207C1C2040201C3C03
:100300004030403C44281028444C9090907C4464F9
:10031000544C44000836410000007700000041368C
:10032000080002010204023C2623263C1EA1A16112
:10033000123A4040207A3854545559215555794144
:100340002154547841215554784020545579400C1B
:100350001E527212395555555939545454593955FC
:100360005454580000457C410002457D420001453F
:100370007C40F0292429F0F0282528F07C545545AC
:10038000002054547C547C0A097F4932494949323F
:100390003248484832324A4848303A4141217A3A54
:1003A00042402078009DA0A07D39444444393D401E
:1003B00040403D3C24FF2424487E4943662B2FFCCB
:1003C0002F2BFF0929F620C0887E09032054547979
:1003D000410000447D413048484A32384040227A4A
:1003E000007A0A0A727D0D19317D2629292F2826C7
:1003F0002929292630484D402038080808080808CF
:100400000808382F10C8ACBA2F102834FA00007B27
:10041000000008142A142222142A1408950022002D
:1004200095AA005500AAAA55AA55AA000000FF00E7
:10043000101010FF00141414FF001010FF00FF1024
:1004400010F010F0141414FC001414F700FF000056
:10045000FF00FF1414F404FC141417101F10101FD5
:10046000101F1414141F00101010F0000000001FC3
:10047000101010101F10101010F010000000FF10CE
:100480001010101010101010FF10000000FF1400CA
:1004900000FF00FF00001F10170000FC04F41414FC
:1004A0001710171414F404F40000FF00F7141414C8
:1004B00014141414F700F7141414171410101F1048
:1004C0001F141414F4141010F010F000001F101F6B
:1004D0000000001F14000000FC140000F010F010D9
:1004E00010FF10FF141414FF141010101F00000050
:1004F00000F010FFFFFFFFFFF0F0F0F0F0FFFFFF54
:100500000000000000FFFF0F0F0F0F0F38444438AA
:10051000447C2A2A3E147E02020606027E027E02E5
:1005200063554941633844443C04407E201E200604
:10053000027E020299A5E7A5991C2A492A1C4C7241
:1005400001724C304A4D4D303048784830BC625AC8
:10055000463D3E494949007E0101017E2A2A2A2A58
:100560002A44445F444440514A444040444A514034
:100570000000FF0103E080FF000008086B6B0836F5
:1005800012362436060F090F060000181800000066
:100590001010003040FF0101001F01011E00191D55
:1005A0001712003C3C3C3C0000000000F0F89C8E20
:1005B0008783878E9CF8F00000FEFF03030303038C
:1005C000070EFCF80000FEFF0303030303070EFC05
:1005D000F80000FFFF00000000000000FFFF000027
:1005E000FEFF8383838383C7EE7C380000F8FC0E14
:1005F00007030303070EFCF800003F7FE0C0808084
:10060000C0E07F3FFFFF01010101010101FFFF0089
:1006100000FFFF0C0C0C0C1C3E77E3C100007FFFB9
:10062000C0C0C0C0C0E0703F1F00001F3F70E0C0EE
:10063000C0C0E0703F1F00007FFFC1C1C1C1C1E366
:10064000773E1C00001F3F70E0C0C0C0E0703F1F3D
:10065000000000000001FFFF01000000D5F08D1434
:10066000A1C881CFD9F1AF20007C7C7C7C7C7C7CD4
:10067000007C7C7C00564F4C207C00415558004348
:10068000482000080B0002020201000904000001DA
:1006900002020000052400100105240101010424C8
:1006A0000206052406000107058103100040090425
:1006B0000100020A000000070502024000000705D1
:1006C00083024000000403090412010002EF02014A
:1006D00040412336800001010203014172647569C3
:1006E0006E6F204C4C430041726475696E6F204CF4
:1006F000656F6E6172646F00830C11241FBECFEFB3
:10070000DAE0DEBFCDBF11E0A0E0B1E0E0E6F2E26A
:1007100002C005900D92A234B107D9F725E0A2E4FA
:10072000B1E001C01D92A93EB207E1F713E0CDE7A9
:10073000D3E004C02197FE010E942311CC37D107DA
:10074000C9F70E94C40C0C942E110C9400008091E7
:100750004F01089580E0E2E7F1E081118FEF00247E
:1007600081938193819381930394D1F70895E2E774
:10077000F1E0A0E0B8E000800EBC8111012C1197DF
:10078000A0FDFDCF0192B9F70DB408959091DC055D
:10079000982329F49091DB05982381E009F480E007
:1007A0000895FC0180917101882311F13FB7F894FD
:1007B00082E08093E9002091F200822F90E01816E9
:1007C000190614F481E090E0882339F0289844E673
:1007D000409370014091F1004083222339F0209131
:1007E000F200211103C02BE62093E8003FBF0895DB
:1007F0008FEF9FEF08952FB7F89483E08093E9007F
:100800009091E800892F807295FF04C09091F200CA
:1008100080E4891B2FBF08958091680181110DC06C
:1008200082E08093640184E0809365011092670107
:100830001092660181E08093680184E691E008955A
:10084000CF93DF931F92CDB7DEB76983DC01ED91C3
:10085000FC910280F381E02D41E050E0BE016F5F2A
:100860007F4F09950F90DF91CF91089583E080939A
:10087000E9008091F200882319F08AE38093E80070
:1008800008950E94FB0390E00895CF93DF931F9299
:10089000CDB7DEB7FC018485958597FD08C02FEFA5
:1008A0003FEF358724870F90DF91CF910895CE01D8
:1008B00001960E94D103019719F4898190E0F3CF4A
:1008C0008FEF9FEFF0CF0F931F93CF93DF931F9284
:1008D000CDB7DEB78C01FC018485958597FF0BC0F1
:1008E000CE0101960E94D103019771F4898190E0B5
:1008F000F80195878487F801848595850F90DF91AD
:10090000CF911F910F9108958FEF9FEFF1CFFC01D1
:100910008485958597FD0BC09FB7F89482E08093FE
:10092000E9008091F2009FBF90E0019608959FB783
:10093000F89482E08093E9008091F2009FBF90E0FC
:10094000089540915E0150915F0120915C013091CA
:100950005D0142175307B4F49091E8009570E1F3FC
:100960009091E80092FD19C08093F10080915E01A2
:1009700090915F0101968F739927892B19F48EEF5F
:100980008093E80080915E0190915F0101969093C1
:100990005F0180935E0181E0089580E00895DF9219
:1009A000EF92FF920F931F93CF93DF93D82E8A017C
:1009B000EB017B01E40EF51ECE15DF0559F0D7FEE5
:1009C00012C0FE0184910E94A10421968111F4CFEE
:1009D0000FEF1FEFC801DF91CF911F910F91FF9093
:1009E000EF90DF9008958881EECF0F931F93CF9300
:1009F000DF931F92CDB7DEB782E0898342E450E0F7
:100A000063E876E080E80E94CF040E940C04DC01D9
:100A100012960D911C910115110589F0D801ED91E7
:100A2000FC910280F381E02DBE016F5F7F4FC80112
:100A3000099597FD04C0F80100851185ECCF8981E7
:100A40000F90DF91CF911F910F910895615030F079
:100A50002091F100FC0120830196F8CF289884E6CC
:100A6000809370010895AF92BF92CF92DF92EF9280
:100A7000FF920F931F93CF93DF936C017B018B0148
:100A8000040F151FEB015E01AE18BF08C017D10798
:100A900059F06991D601ED91FC910190F081E02D22
:100AA000C6010995892B79F7C501DF91CF911F9177
:100AB0000F91FF90EF90DF90CF90BF90AF9008958F
:100AC0003FB7F89480914B0190914C01A0914D015A
:100AD000B0914E0126B5A89B05C02F3F19F0019695
:100AE000A11DB11D3FBFBA2FA92F982F8827BC0188
:100AF000CD01620F711D811D911D42E0660F771FB0
:100B0000881F991F4A95D1F708958F929F92AF92AF
:100B1000BF92CF92DF92EF92FF926B017C010E9415
:100B200060054B015C01C114D104E104F104B9F08A
:100B30000E946005681979098A099B09683E73401B
:100B40008105910580F321E0C21AD108E108F1087E
:100B500088EE880E83E0981EA11CB11CE4CFFF90A4
:100B6000EF90DF90CF90BF90AF909F908F900895BF
:100B70008F929F92AF92BF92CF92DF92EF92FF92AD
:100B80000F931F93CF93DF936C017B018A018091B8
:100B90001401882309F45CC080917101882309F451
:100BA00057C08091630180FF05C08091E0008260A2
:100BB0008093E000E801B12C8AEFA82E93E0892E03
:100BC0002AE3922E209711F4BB20D9F10E94FB0357
:100BD00081110AC0AA94AA20D9F161E070E080E0F6
:100BE00090E00E948505EECF8C171D0611F00CF0E9
:100BF0008C2F9FB7F8948092E9002091E80025FDA2
:100C000002C09FBFDFCF282F30E0C21BD30BF701FC
:100C1000815020F041914093F100FACFE20EF31E93
:100C2000BB2021F09092E800B12CEBCF8091E8003E
:100C300085FDE7CF9092E800BB24B394209709F399
:100C4000F3CF5D9884E680936201101611063CF0A4
:100C500081E090E0F6019383828310E000E0C80118
:100C6000DF91CF911F910F91FF90EF90DF90CF9088
:100C7000BF90AF909F908F90089520915901E0917F
:100C80005701F0915801CF0102969093580180933B
:100C90005701222319F085919491089580819181C3
:100CA0000895CF92DF92EF92FF92CF93DF930E944D
:100CB0003D06811520E8920791F4809171008D7FA7
:100CC00080937100109291004698479810925401B9
:100CD000DF91CF91FF90EF90DF90CF90089521E0CA
:100CE00020935401813020E8920751F480915501FE
:100CF0009091560190935801809357010E943D06B0
:100D000097FD05C020914301222309F454C020918E
:100D10004201211150C021E020934401EC01DF7712
:100D2000209709F04BC081E08093450146983FE948
:100D3000C32E3FE0D32EE12CF12CCAEFD0E0E0919E
:100D4000D005F091D1050995811103C081E0809310
:100D5000450180914401882329F080914501882331
:100D600009F43FC047980E943D060097F1F19C01AD
:100D7000DE010E941411DC01CB0129E0B595A79595
:100D8000979587952A95D1F7109290002AE02093A5
:100D90009100D0929900C092980080934601909360
:100DA0004701A0934801B09349018091710082608E
:100DB000809371008DCF10924401B0CF9E0150E01E
:100DC00040E060E472E48FE090E00E94D31069019B
:100DD0007A0181E0C81AD108E108F10810924501B2
:100DE000AECF4699BFCF479ABECF8FEF9FEFDC01C2
:100DF000CBCF2D9A0895BC0190E080E00C9485053E
:100E00008FB18095807F669B88601C9B846008956D
:100E100020E191E061FD94E060FD990F62FD929503
:100E2000687F269FD0011124A80FAE58BE4F8C9129
:100E300040FF03C0892B8C93089590958923FBCFA5
:100E40002F923F924F925F926F927F928F929F92DA
:100E5000AF92BF92CF92DF92EF92FF920F931F93C8
:100E6000CF93DF93CDB7DEB728970FB6F894DEBFE8
:100E70000FBECDBF9E838D836A3061F5DC01559630
:100E80008C91B8E08B9F90011124ED81FE818189C6
:100E90009289820F931F928B818B108A178681E033
:100EA00090E028960FB6F894DEBF0FBECDBFDF915D
:100EB000CF911F910F91FF90EF90DF90CF90BF9057
:100EC000AF909F908F907F906F905F904F903F90EA
:100ED0002F9008956D3019F32D813E8138872F832F
:100EE000D9011F960D911C915097003811050CF0F7
:100EF0007CC05196AD90BC90B0E4AB16B1040CF040
:100F000074C0F901258825E0C801229E800D911D3D
:100F10001124181619060CF068C0622C712CC3013C
:100F200033E0880F991F3A95E1F78A0D9B1D18163B
:100F300019060CF05AC0F489FB83AF81B88553962B
:100F4000BC91BC83629FB0011124FB01E455FF4FAB
:100F50002F011982F2018491F981F53009F480E0C2
:100F6000450128E02A83A82FB0E0BE83AD833C80F2
:100F700080FF3B80311004C0BB81EC81BE17F9F0CB
:100F800078018E2D801B8215D0F4D12CC12CC21477
:100F900090F4F0E8EF16F10450F4B601680D791DF5
:100FA0006034710520F4432DC7010E9408072FEF1C
:100FB000C21AD20AECCF3FEFE31AF30AE2CF8D81D7
:100FC0009E81959587959A8191509A83860C971C5E
:100FD0009111C9CFA981AF5FA983BFEF4B1A5B0AFB
:100FE000060D171DA63009F0B5CFEF81F8852589CC
:100FF000422F50E087859089F6E02F9F800D911D4C
:101000001124AF81B88550969C938E931F97569666
:101010002C915697222309F442CF6AEF6403900182
:10102000659F300D112420583F4F281739070CF0C9
:1010300036CFED91FC9111970190F081E02D6AE09F
:10104000CD0109952CCF0F931F93CF93DF938C0184
:10105000D0E0C0E0F801EC0FFD1F6491662341F081
:1010600082ED95E00E942007892B11F02196F2CFA6
:10107000CE01DF91CF911F910F91089508950895AA
:1010800090E080E00895409100015091010160914D
:10109000020170910301DB01CA0181709927AA271F
:1010A000BB27B095A095909581959F4FAF4FBF4FAF
:1010B00081709927AA27B07D7695679557954795B2
:1010C00084279527A627B7278093000190930101D5
:1010D000A0930201B093030108958F929F92AF9263
:1010E000BF920F931F93CF93DF93CDB7DEB7A19736
:1010F0000FB6F894DEBF0FBECDBF19A2423008F480
:101100004AE08E010F5D1F4F842E912CB12CA12C33
:10111000A50194010E94F210E62FB901CA01EA303C
:1011200044F5E05DD801EE938D01232B242B252B74
:1011300079F790E080E0109769F0FD0101900020C0
:10114000E9F73197AF014A1B5B0BBD0182ED95E0DA
:101150000E943305A1960FB6F894DEBF0FBECDBF37
:10116000DF91CF911F910F91BF90AF909F908F9083
:101170000895E95CD7CF0C94BD100E9429111F92ED
:101180000F920FB60F9211248F939F938091E100DD
:101190009091E100937F9093E10083FF0FC0109244
:1011A000E90091E09093EB001092EC0092E39093B1
:1011B000ED001092710198E09093F00082FF22C040
:1011C00093E09093E9009091F200992319F09AE34B
:1011D0009093E80090916201992341F0909162010F
:1011E000915090936201911101C05D9A90917001AC
:1011F000992341F090917001915090937001911159
:1012000001C0289A84FF18C08091E2008E7E816020
:101210008093E2008091E1008F7E8093E1008091D5
:1012200063018E7E8061809363019F918F910F9007
:101230000FBE0F901F90189580FFF7CF8091E200AE
:101240008E7E80618093E2008091E1008E7E8093AB
:10125000E100809163018E7E8160E5CF1F920F9245
:101260000FB60F921124CF92DF92EF92FF920F935D
:101270001F932F933F934F935F936F937F938F931E
:101280009F93AF93BF93EF93FF93CF93DF93CDB72C
:10129000DEB76C97DEBFCDBF1092E9008091E80009
:1012A00083FF25C068E0CE0145960E94260582EFA7
:1012B0008093E8008D8987FF39C09091E80090FF06
:1012C000FCCF982F907609F034C19E894F89588DB4
:1012D0002F89F88C911131C0803861F580916101BE
:1012E0008093F1001092F1008EEF8093E8006C96ED
:1012F0000FB6F894DEBF0FBECDBFDF91CF91FF9147
:10130000EF91BF91AF919F918F917F916F915F917D
:101310004F913F912F911F910F91FF90EF90DF9090
:10132000CF900F900FBE0F901F9018959EEF909347
:10133000E800C7CF1092F100D5CF913059F4811158
:10134000D3CF4130510581F6809161018D7F80932B
:101350006101CACF933049F48111C6CF41305105A4
:1013600019F6809161018260F2CF953041F480914D
:10137000E80080FFFCCF20682093E300B5CF9630D3
:1013800009F0A9C00B8D1C8D22E01092E90010928B
:101390005F0110925E01F2122EC010925D01109258
:1013A0005C010E94F5041F8299E09983FA8291E022
:1013B0009E8390EA98879AEF998720915E013091F9
:1013C0005F01275F3F4F3C832B838D831092E900A1
:1013D00010925F0110925E0110935D0100935C0119
:1013E00049E050E0BE016F5F7F4F80E00E94CF0474
:1013F0000E94F50479CF10935D0100935C010E9477
:101400000C04DC0112960D911C910115110509F4D3
:1014100051C1D801ED91FC910480F581E02DBE0110
:101420006B5E7F4FC8010995009709F03EC1F80136
:1014300000851185EACFF3E0FF120EC08F89882363
:1014400009F440C0823061F440E860E187EE96E044
:101450000E940B0C811148CF81E28093EB0047CFB3
:10146000813029F440E86BE08BED96E0F1CF8330DA
:1014700099F70E940C04DC011296ED90FC908E010D
:101480000F5F1F4F6801E114F10479F0D701ED916E
:10149000FC910680F781E02DB801C7010995080F7E
:1014A000111DF701E084F184EECFD8011C92F60102
:1014B00001900020E9F73197BF016C197D0940E0E8
:1014C000C601C6CF65EC76E0FB01449150E080E8B0
:1014D0000E94CF0409CF973009F4BECF983021F491
:1014E00081E08093F10000CF993009F0FDCE837048
:1014F00009F0B2CFE6E1F1E081E031E096E321913D
:10150000222371F08093E9003093EB00DF01119703
:101510002C912093EC009093ED008F5F873079F74A
:101520008EE78093EA001092EA008F898093710120
:10153000DBCE8B8D9C8D1092E90010925F01109292
:101540005E0190935D0180935C01898D811192C051
:101550008E899D89913A49F4813209F07DCF47E027
:1015600050E06DE071E080E0B3CF913209F074CFCC
:10157000833269F48F89988DB0E0A0E080930901EF
:1015800090930A01A0930B01B0930C01ADCE803271
:1015900069F48091E80082FFFCCF67E08DE091E084
:1015A0000E9426058BEF8093E8009ECE823209F0E0
:1015B0009BCE8F8980931401EEEFFFE78591949184
:1015C0008B3F9C4D51F1E0E0F8E080910D0190914E
:1015D0000E01A0910F01B0911001803B9440A10534
:1015E000B105F1F48091140180FD1AC0EE3F8AE04C
:1015F000F80789F587E797E79183808380916000FA
:101600008093600188E19BE00FB6F894A8958093E1
:1016100060000FBE9093600067CEEEEFFAE0D5CF8A
:10162000808191818737974709F05ECEA895809198
:101630006000886180936000809160018093600009
:10164000EE3F2AE0F20789F08091FE0A9091FF0AAE
:101650009183808349CE808191818737980751F2A9
:101660009093FF0A8093FE0AC5CF1092FF0A109252
:10167000FE0A3ACE0E940C04DC0112960D911C91D8
:101680000115110509F4E8CED801ED91FC91019006
:10169000F081E02DBE016B5E7F4FC801099581117D
:1016A00023CEF80100851185EBCF181619060CF42E
:1016B0001BCED2CEF1E0FF12BECE69EC76E004CFB5
:1016C0001F920F920FB60F9211242F933F938F9377
:1016D0009F93AF93BF938091500190915101A0913E
:1016E0005201B091530130914A0123E0230F2D376D
:1016F00058F50196A11DB11D20934A018093500118
:1017000090935101A0935201B093530180914B01EA
:1017100090914C01A0914D01B0914E010196A11DF7
:10172000B11D80934B0190934C01A0934D01B09358
:101730004E01BF91AF919F918F913F912F910F904B
:101740000FBE0F901F90189526E8230F0296A11D3B
:10175000B11DD2CF1F920F920FB60F9211242F936B
:101760003F934F935F936F937F938F939F93AF9329
:10177000BF93EF93FF938091460190914701A09111
:101780004801B0914901892B8A2B8B2B09F440C069
:101790008091450181110BC088B190E4892788B9F7
:1017A00080914401882319F088B1805888B98091CC
:1017B000460190914701A0914801B0914901181646
:1017C00019061A061B069CF4809146019091470168
:1017D000A0914801B09149010197A109B1098093F5
:1017E000460190934701A0934801B0934901FF91AE
:1017F000EF91BF91AF919F918F917F916F915F9189
:101800004F913F912F910F900FBE0F901F90189501
:101810000E945106ECCFEF92FF920F931F93CF934C
:10182000DF93F82E192FE62E042F81E0860F880F04
:101830000E94A10483E00E94A104CF2DD12FEC0EC1
:10184000FD2EF11CCE15DF05B9F007FF13C0FE0118
:1018500084910E94A104182F80E00E94A10481239A
:1018600021968111EFCFDF91CF911F910F91FF90C2
:10187000EF9008958881EDCF81E0F5CF0F931F930E
:10188000CF93DF938C0181E090E00E94BB0880FF42
:1018900032C08AE090E00E94BB089FEF980F9E3F05
:1018A00050F522E330E0D80150963C932E931F97D9
:1018B00028E330E052963C932E935197CBE0D0E052
:1018C000D801ED91FC910190F081E02D682FC801C5
:1018D0000995CE010E94BB082196C131D10581F73F
:1018E00080E00E94B70388EE93E0DF91CF911F91D3
:1018F0000F910C94FB06DF91CF911F910F910895EA
:1019000004970C943E0CE2E7F5E01382128288EE15
:1019100093E0A0E0B0E084839583A683B78380E260
:1019200091E0918380838FEF9FEF95878487E2ED2D
:10193000F5E0138212821186128680E18387108679
:101940001782158682E391E09183808380E491E0A1
:1019500095838483108A1786128A118A81E0838B8B
:10196000148A858B168A87EA93E09093D105809339
:10197000D00580E090E89093CF058093CE054698FF
:101980003E9A47983F9A0895789484B5826084BDC2
:1019900084B5816084BD85B5826085BD85B5816073
:1019A00085BD80916E00816080936E0010928100F1
:1019B00080918100826080938100809181008160AC
:1019C000809381008091800081608093800080916D
:1019D000910082608093910080919100816080935A
:1019E0009100809190008160809390008091C1006F
:1019F00084608093C1008091C10082608093C100A7
:101A00008091C10081608093C1008091C30081609A
:101A10008093C3008091C00082608093C000809159
:101A2000C20081608093C20080917A0084608093BC
:101A30007A0080917A00826080937A0080917A00A7
:101A4000816080937A0080917A00806880937A0028
:101A50001092710110926101109263018091D70080
:101A600081608093D70080EA8093D80089B5806137
:101A700089BD89B5826089BD09B400FEFDCF61E0F2
:101A800070E080E090E00E9485058091D8008F7C16
:101A900080618093D8008091E000807F8093E00097
:101AA0008091E1008E7E8093E1008DE08093E200E2
:101AB000559A209A81EC80937C0085B1806F85B91E
:101AC00084B1877E84B984B1876E84B95E9A5F9849
:101AD0008AB1806D8AB9769A6E9881B3806F81BB26
:101AE000899880B38D7080BB80E58CBD81E08DBD11
:101AF00085E090E00E94FB065F9A85E090E00E94FE
:101B0000FB065E985C98ECE5F6E089E696E02491A9
:101B10002EBD00000DB407FEFDCF31968E179F0736
:101B2000B1F75C9A81E880936400809165008160E0
:101B30008093650080E00E94B7030E94000787FF42
:101B400015C05C9885EA8EBD00000DB407FEFDCF80
:101B50005C9A2E982F982D988091640080628093D3
:101B6000640081E083BF889513BEFCCF0E9400070C
:101B700082FF48C02D980E94000784788438E1F4E1
:101B80000E94F90688EC90E00E94FB062F9882E004
:101B900090E00E94BD108F3F29F06FEF82E090E04F
:101BA0000E94C51084EF91E00E94FB062F9A0E94CC
:101BB000000784788438D9F30E9400078471843147
:101BC000E1F40E94F90688EC90E00E94FB062E9852
:101BD00082E090E00E94BD10882329F060E082E05E
:101BE00090E00E94C51084EF91E00E94FB062E9ABF
:101BF0000E94000784718431D9F388EC90E00E9440
:101C0000FB06B4CF0E94F90682E090E00E94BB0878
:101C1000882309F45BC03E9A3F9A81E080934F018C
:101C200081E090E00E94BB08382F3470932E81FF32
:101C30000EC031112E98C0EFDFEF08E010E00E94D7
:101C4000000786FF48C02E9A2F9A0E94F90682E369
:101C500090E00E94FB060E9400078111F8CF80E10E
:101C60008093DD050E94AA031092E4051092E3051B
:101C70001092E2051092E10562E0462E512C42ECF2
:101C8000A42E45E0B42E5AE0652E712C8FB7F8943F
:101C90004091500150915101609152017091530156
:101CA0008FBF8091DE05F42FF81B8F2F9091DF05F9
:101CB000992309F49FC0F093E0051092DF0580E0BE
:101CC00090E0892B19F30E940000D9CF10924F01A8
:101CD0003E983F98A5CF992029F0C430D10511F442
:101CE0002E9A2F9881E00E94B7039E01D7FF04C06F
:101CF000222733272C1B3D0B27703327CE01D7FD1E
:101D00000796E3E095958795EA95E1F7D7FF05C03B
:101D10000197A801421B530B9A01AC015695542F11
:101D20004427579547954E585E4FF12CE12C3801CA
:101D3000621A730A8F3F6FEF9607B4F1DA01AC565F
:101D4000BF4F6A0170E060E0F701E455FA4F5F01B0
:101D50008F3F980779F0F501E60FF71FE491F0E067
:101D60002F01022E01C0440C0A94EAF7F601848880
:101D70004828448A2115310571F0F501E60FF71F57
:101D8000E491F0E0062C02C0F595E7950A94E2F79D
:101D9000FC91EF2BEC936F5F7F4F1196FFEFCF1A03
:101DA000DF0A68357105A1F6019668E5E60EF11CBB
:101DB00040585F4FE0EBEE16F10409F0BBCF80E036
:101DC0000E94B7038FE090E00E94FB062196C93184
:101DD000D10509F034CF992011F02F9A2D9880E980
:101DE00091E00E94FB060E94F90682ED95E00E94B8
:101DF0003E0C2DCF9091DD05F91748F48F5F8917C0
:101E000008F05DCF81E083BF889513BE58CF81E095
:101E10008093DF054093DE058091D9059091DA0526
:101E200001969093DA058093D9058091DB05809324
:101E3000DC050E9400078093DB0580910801882360
:101E400009F432C180915B0118167CF5809106017E
:101E5000882359F180910701863438F58091540127
:101E6000811123C00E94430890E090582091710096
:101E70002D7F2093710010925901B0925801A092C9
:101E80005701B0925601A09255019093C3058093DB
:101E9000C2057092C5056092C40580E090E89093F9
:101EA000C7058093C6050E9451068091D9053AEA7C
:101EB000F32E80FD02C025E5F22ED090070136E416
:101EC0003D1508F4F12CD0E0C0E08E0108571E4FFC
:101ED00098E0E92EC09006018FEFC1100E944308E0
:101EE0008F21F8018083EA9400581F4FE110F2CF50
:101EF0002196C335D10549F7DD20D1F145E450E005
:101F00005093E2054093E1055092E4054092E305C9
:101F1000CC2009F4B6C08FE796E00E942308809198
:101F200005018A302CF460E282ED95E00E942007E2
:101F3000C09005010C2C000CDD08EE08FF084AE0FB
:101F4000C701B601F7FE0DC06DE282ED95E00E947B
:101F5000200766277727CB016C197D098E099F0919
:101F60004AE00E946D08809107018150809307012B
:101F7000809104018823F1F088E190E09093E205DC
:101F80008093E105E6E3F0E0F093E405E093E305F8
:101F900085E796E00E94230880915B01813009F07B
:101FA00075C081E796E00E9423088091040181506A
:101FB0008093040180E80E94C603882359F0809131
:101FC0005B0118160CF468C08F5F80935B0180E59D
:101FD0008093040180E10E94C603882359F0809118
:101FE0005B0182300CF45AC0815080935B0180E524
:101FF0008093040180E40E94C603882379F08091D5
:102000000601882341F0809105018D300CF048C015
:102010008F5F8093050180E58093070180E20E9435
:10202000C603882371F080910601882339F08091DE
:1020300005018330BCF181508093050180E58093D8
:10204000070188E00E94C603882349F080910601B9
:1020500091E089278093060180E58093070184E061
:102060000E94C603882349F08091080191E08927E6
:102070008093080180E580935A0180E00E94B703B5
:102080001ECE8BE796E00E9423086DCF823009F0C8
:102090008CCF89E696E087CF82E097CF80E0A5CF0E
:1020A00082E0B7CF8DE0C8CF0E94AA031092E4056A
:1020B0001092E3051092E2051092E10530905A016A
:1020C000332009F44BC0F6E4F315F0F52AEB230DA9
:1020D000022F000F020F000FC22ECC0CCC0CCC0C28
:1020E0003DEF32037001112440E2E40EF11CC0E127
:1020F000D0E0C21BD109CC0FDD1FCC0FDD1FCC0EF1
:10210000DD2ED11C0E0D1F2D111DCC15DD05E4F4A7
:102110004701F7FE02C0912C812CC8010134110542
:1021200014F080E490E08816990664F4C038D10574
:1021300028F441E0B401CE010E9408075FEF851A40
:10214000950AEBCF2196E1CF41E060E270E080E4B8
:1021500090E00E9408073A9430925A0184E00E946D
:10216000C603882309F489CF81E08093080180E5C4
:10217000809307018093040180CFF999FECF92BD2F
:1021800081BDF89A992780B50895262FF999FECF39
:102190001FBA92BD81BD20BD0FB6F894FA9AF99A84
:1021A0000FBE01960895052E97FB1EF400940E9421
:1021B000EA1057FD07D00E94F21007FC03D04EF43E
:1021C0000C94EA1050954095309521953F4F4F4F14
:1021D0005F4F089590958095709561957F4F8F4FD3
:1021E0009F4F0895A1E21A2EAA1BBB1BFD010DC033
:1021F000AA1FBB1FEE1FFF1FA217B307E407F507B7
:1022000020F0A21BB30BE40BF50B661F771F881F92
:10221000991F1A9469F760957095809590959B0128
:10222000AC01BD01CF010895A29FB001B39FC001D1
:10223000A39F700D811D1124911DB29F700D811DF2
:102240001124911D0895EE0FFF1F0590F491E02DCC
:10225000099481E090E0F8940C942E11F894FFCF4B
:10226000010000005003015001FFFFFFFF00E100EB
:10227000000000000000C18081000000000000009C
:102280002004B805410436048704450463040000B3
:1022900000002007330540083F083E0CFCFF00000B
:0222A000800CB0
:00000001FF
